:020000020000FC
:020000006FC0CF
:02000800189549
:0200160002C026
:10001A000DC00F931F930FB716B31C7019F411E09C
:10002A00109360000FBF1F910F9118950F931F93A4
:10003A002F933F934F935F935FB74091670045308B
:10004A000CF403C0442740936700403081F493982E
:10005A00949895980EF002C00BE002C000916500DA
:10006A00002311F0929A01C0929850D305D24130E0
:10007A0081F4929894989598009164003091650063
:10008A00032B11F0939A01C09398009164003ED318
:10009A00F3D1423059F4929893989598949A009192
:1000AA00630034D3002D0F77002EE6D1433041F49C
:1000BA00929893989498959A0091660027D3DCD1E8
:1000CA004395409367005FBF5F914F913F912F9196
:1000DA001F910F9118950FED0DBF0FE701BB01EEB0
:1000EA0007BB0CE108BB02E000BF05E003BF03E267
:1000FA0006BF00E20BBF0CE100BD03E309B900E053
:10010A0002B908E00AB906E003B91124109267009F
:10011A0000E00093600004E0302EEAD0042D0031A4
:10012A0011F09CD014C000E0302EE2D040926B0057
:10013A0001E0302EDDD040926C0002E0302ED8D0A3
:10014A0040926D0003E0302ED3D040926E0000271B
:10015A00009368000093690000EF00936A000FEFB4
:10016A0000937100662428D100916F00083209F4C7
:10017A0005C012E010936000DBD201C0D2D280E049
:10018A0090E000916000003051F420916A002093C1
:10019A00660003D1A1D2B4D011E019BF41D0013019
:1001AA0009F4A6D1023069F71BE01093630010939B
:1001BA006400109365001093660011E019BFE1CF47
:1001CA00EE24FF1841E1001F111F4A9509F4089512
:1001DA00EE1CFF1CE21AF30A20F4E20EF31E8894C6
:1001EA00F2CF0894F0CFFF1829E0001F2A9509F4EE
:1001FA000895FF1CF11A18F4F10E8894F6CF0894AA
:10020A00F4CF5527442760E13695279510F4400F1F
:10021A00511F57954795379527956A95B9F70895C8
:10022A000F931F9300916800502E14D000916A001A
:10023A00502E10D000B30170502E0CD004E0502E76
:10024A0009D00027502E1CE005D01A95E9F71F9116
:10025A000F9108955D9BFECF5CB8089501E000936D
:10026A006B00402E00E0302E36D00CE200936C007A
:10027A00402E01E0302E2FD005E000936D00402E75
:10028A0002E0302E28D001E000936E00402E03E0F9
:10029A00302E21D000E1402E04E0302E1CD00895EB
:1002AA000F9300916B00402E00E0302E14D0009185
:1002BA006C00402E01E0302E0ED000916D00402ED1
:1002CA0002E0302E08D000916E00402E03E0302E5E
:1002DA0002D00F910895F8940F93E199FECF00E0B0
:1002EA000CBB3EBA4DBAE29AE19A0F9178940895FE
:1002FA00F894E199FECF3EBAE09A4DB27894089507
:10030A000F931F932F933F934F935F937F93009184
:10031A006800109169002AE030E073DF022F132F82
:10032A0020916A003327020F131F40916C005091ED
:10033A006B0060916D004F935F937727461B570BB5
:10034A00B42EA52E5F914F917727460F571FD42EB3
:10035A00C52E0EF004C0009510950F5F1F4FB01602
:10036A00A10624F40D151C054CF40FC040916E0033
:10037A00442311F4909801C0909A07C040916E00EE
:10038A00442311F4909A01C090987F915F914F9104
:10039A003F912F911F910F9108951F9361D052E1C0
:1003AA0035E54DEBE0D112D010916800812F109104
:1003BA006900912F1F9108950F9340D103E3802E76
:1003CA0052D1AFE6B0E06ED10F9108950F931F930B
:1003DA002F933F934F9332D170FF3CC00CEC802E89
:1003EA0042D10EEB802E3FD1A8E6B0E05BD1A9E660
:1003FA00B0E058D110916800209169002F93287FAE
:10040A00283F11F0E89407C02F9168941095209521
:10041A001F5F2F4F01C02F91269517952695179587
:10042A002695179526951795309168000EF4319503
:10043A00432F3F70432F330F330F330F440F340FC3
:10044A00369536953695369510936800209369004F
:10045A0030936A004F913F912F911F910F91089508
:10046A000F93ECD070FF06C00CEC802EFCD004E495
:10047A00802EF9D00F9108950F930F920FB800E4D0
:10048A000EB90BE10DB9769BFDCFC09AC0980F90BB
:10049A000F9108950F93B49B01C01CC00091710085
:1004AA00002309F417C000270093710048D1639410
:1004BA00162D143014F435D10DC010E019BF9298DE
:1004CA009398949895986624EBDE32D1969810E02A
:1004DA0010936000B49901C009C000917100002313
:1004EA0009F004C00FEF0093710029D10F9108950C
:1004FA000F931F932F933F934F93062D002309F0D9
:10050A0004C09098969A0DD16394C4DF013029F003
:10051A00023049F1033031F18BC0DED0B29B04C006
:10052A0000C0B39B0AC011C00AD110916D00183CDB
:10053A0009F0139510936D0008C001D110916D0058
:10054A00113009F01A9510936D000F931F930091C3
:10055A006D001AE048DE802F9927F09266001F91FD
:10056A000F9166C03FC0B8D0B29B04C000C0B39B15
:10057A000FC019C0E4D010916C0020916B003AE0D2
:10058A00130F3327231F10936C0020936B000BC0AB
:10059A00D6D010916C0020916B001A502040109315
:1005AA006C0020936B000F931F932F933F9300913E
:1005BA006C0010916B00212F207811F4E89405C08B
:1005CA006894009510950F5F1F4F2AE030E0F8DD20
:1005DA00802F912F0AE0009366003F912F911F917F
:1005EA000F9126C0E894B29B04C000C0B39B06C01A
:1005FA0009C0A5D011E010936E0004C0A0D010E08D
:10060A0010936E001127812F912F112710936300E9
:10061A00109364001093650020916E00222309F064
:10062A0004C01CE01093660003C01DE0109366002E
:10063A004F913F912F911F910F910895F894B99A74
:10064A0033E04EEB8CD0B99830E04AE888D005D038
:10065A0033E042E384D078940895B19B716002C07C
:10066A00B1997E7F0895F8940F931F93082D18E08F
:10067A00069508F448F0B99A30E046E770D0B99880
:10068A0030E042E16CD008C0B99A30E04AE067D065
:10069A00B99830E04EE763D01A9551F71F910F9140
:1006AA0078940895F8940F931F93002718E00695FD
:1006BA00B99A30E04AE053D0B99830E040E14FD0DF
:1006CA00B199006830E04CE64AD01A9581F70C934C
:1006DA001F910F91789408950F935F9353E0A3E6C7
:1006EA00B0E08093610090936200009161001091E4
:1006FA0062002AE030E064DDED920093610010931D
:10070A0062005A9591F75F910F9108950F931F9385
:10071A00EAE7F7E01127E00FF11F04901F910F910C
:10072A000895C59A53E039EA4DE71DD0C598089552
:10073A00C59A5CE034E34DEF16D0C59808950F933F
:10074A001F932F932AE01FEF0FEF0A95F1F71A95DF
:10075A00D9F72A95C1F72F911F910F91089541500A
:10076A003040E8F70895415030405040E0F708958E
:0E077A00C0F9A4B0999282F880909CBFC68905
:00000001FF
